:1000000012C02AC029C028C027C026C025C024C0CD
:1000100023C022C021C020C01FC01EC01DC01CC0E4
:100020001BC01AC019C011241FBECFEDCDBF10E0F8
:10003000A0E6B0E0E8E2F1E002C005900D92A03643
:10004000B107D9F710E0A0E6B0E001C01D92A036DC
:10005000B107E1F718D066C0D3CF882311F4D99A3D
:1000600001C0D998662311F4D89A01C0D89825E622
:1000700034E08599FECF859BFECFC9010197F1F74A
:10008000859BF7CF08950F931F9383E08ABB17BA20
:1000900011BA87E08BBB80E488BB8FE582BBB69941
:1000A0000BC0809B02C0D99A01C0D998819B02C025
:1000B000D89AF5CFD898F3CF81E060E0CEDF10E09A
:1000C00000E001C016E080B390E0012E02C09595DB
:1000D00087950A94E2F780FF05C080E060E0BDDF0D
:1000E000009503C080E061E0B8DF1F5F153051F379
:1000F000173048F3B09904C080E061E0AEDF04C07F
:1001000080E060E0AADF0095B19B05C080E060E080
:10011000A4DF009503C080E061E09FDF80E0602FF6
:080120009CDFBDCFF894FFCF76
:00000001FF
